:100000000C9428030C9450030C9450030C9450034C
:100010000C9450030C944B090C9450030C94500313
:100020000C9450030C9450030C9450030C94500304
:100030000C9450030C9450030C9450030C945003F4
:100040000C94420F0C9450030C9450030C945003E6
:100050000C9450030C9450030C9450030C945003D4
:100060000C9450030C945003F109F609FB09000AA3
:10007000050A0A0A0F0A140A190A1E0A230A0000AE
:100080000000003E5B4F5B3E3E6B4F6B3E1C3E7C78
:100090003E1C183C7E3C181C577D571C1C5E7F5E26
:1000A0001C00183C1800FFE7C3E7FF0018241800E5
:1000B000FFE7DBE7FF30483A060E2629792926407C
:1000C0007F050507407F05253F5A3CE73C5A7F3EA8
:1000D0001C1C08081C1C3E7F14227F22145F5F003A
:1000E0005F5F06097F017F006689956A60606060D6
:1000F0006094A2FFA29408047E040810207E2010C1
:1001000008082A1C08081C2A08081E101010100CC9
:100110001E0C1E0C30383E3830060E3E0E06000017
:1001200000000000005F00000007000700147F14BB
:100130007F14242A7F2A122313086462364956202A
:10014000500008070300001C2241000041221C004F
:100150002A1C7F1C2A08083E08080080703000080E
:1001600008080808000060600020100804023E51E2
:1001700049453E00427F4000724949494621414974
:100180004D331814127F1027454545393C4A4949DB
:100190003141211109073649494936464949291E45
:1001A0000000140000004034000000081422411434
:1001B00014141414004122140802015909063E4186
:1001C0005D594E7C1211127C7F494949363E4141AE
:1001D00041227F4141413E7F494949417F09090907
:1001E000013E414151737F0808087F00417F410073
:1001F0002040413F017F081422417F404040407F22
:10020000021C027F7F0408107F3E4141413E7F096E
:100210000909063E4151215E7F09192946264949AF
:10022000493203017F01033F4040403F1F204020EF
:100230001F3F4038403F63140814630304780403ED
:100240006159494D43007F4141410204081020009B
:100250004141417F0402010204404040404000030C
:1002600007080020545478407F28444438384444D8
:100270004428384444287F385454541800087E09D0
:100280000218A4A49C787F0804047800447D4000F0
:100290002040403D007F1028440000417F40007C0A
:1002A000047804787C080404783844444438FC1802
:1002B00024241818242418FC7C08040408485454E6
:1002C000542404043F44243C4040207C1C20402013
:1002D0001C3C4030403C44281028444C9090907C7A
:1002E0004464544C4400083641000000770000008C
:1002F0004136080002010204023C2623263C1EA1CE
:10030000A161123A4040207A38545455592155552C
:1003100079412254547842215554784020545579DB
:10032000400C1E527212395555555939545454596E
:1003300039555454580000457C410002457D420027
:1003400001457C407D1211127DF0282528F07C5457
:100350005545002054547C547C0A097F4932494950
:1003600049323A4444443A324A4848303A414121B9
:100370007A3A42402078009DA0A07D3D4242423D15
:100380003D4040403D3C24FF2424487E4943662BA9
:100390002FFC2F2BFF0929F620C0887E090320544B
:1003A0005479410000447D413048484A3238404049
:1003B000227A007A0A0A727D0D19317D2629292FA9
:1003C00028262929292630484D40203808080808C1
:1003D00008080808382F10C8ACBA2F102834FA00C3
:1003E000007B000008142A142222142A1408550045
:1003F000550055AA55AA55AAFF55FF55FF00000004
:10040000FF00101010FF00141414FF001010FF0064
:10041000FF1010F010F0141414FC001414F700FF77
:100420000000FF00FF1414F404FC141417101F1034
:10043000101F101F1414141F00101010F0000000E3
:10044000001F101010101F10101010F010000000EE
:10045000FF101010101010101010FF10000000FFFF
:10046000140000FF00FF00001F10170000FC04F440
:1004700014141710171414F404F40000FF00F714F8
:10048000141414141414F700F7141414171410107F
:100490001F101F141414F4141010F010F000001F9B
:1004A000101F0000001F14000000FC140000F010DA
:1004B000F01010FF10FF141414FF141010101F0080
:1004C000000000F010FFFFFFFFFFF0F0F0F0F0FF82
:1004D000FFFF0000000000FFFF0F0F0F0F0F384459
:1004E000443844FC4A4A4A347E02020606027E022E
:1004F0007E0263554941633844443C04407E201EDB
:100500002006027E020299A5E7A5991C2A492A1C09
:100510004C7201724C304A4D4D303048784830BCF6
:10052000625A463D3E494949007E0101017E2A2A20
:100530002A2A2A44445F444440514A444040444AA1
:1005400051400000FF0103E080FF000008086B6BD2
:10055000083612362436060F090F06000018180058
:1005600000001010003040FF0101001F01011E00BB
:10057000191D1712003C3C3C3C000000000000002C
:100580000008000201000003040700000000000052
:10059000000000000000240027002A0001020408D7
:1005A00010204080010204081020010204081020DD
:1005B00000000000250028002B00040404040404AB
:1005C000040402020202020203030303030304E021
:1005D00010021C07123732292D29252B390001035F
:1005E00010E110031D07062E2C292D2E2E373F005B
:1005F00000021013800A298064022A040000007F90
:100600002B040000009F0F0180961180FFB10301B1
:100610002C2DB203012C2DB306012C2D012C2DB451
:100620000107C003A20284C101C5C2020A00C302BD
:100630008A2AC4028AEEC5010E20003601C83A019A
:1006400005000000002300260029000082127C1211
:1006500011241FBECFEFD8E0DEBFCDBF22E0A6E061
:10066000B2E001C01D92AD35B207E1F712E0A0E0A3
:10067000B1E0E2EEF4E302C005900D92A630B107BE
:10068000D9F713E0C7E2D3E004C02197FE010E942E
:100690005218C632D107C9F70E9416130C94641A77
:1006A0000C9400000895FC016370658B8481958132
:1006B00026813781613039F0633029F09187808756
:1006C000338722870895318720879387828708950B
:1006D0002F923F924F925F926F927F928F929F9252
:1006E000AF92BF92CF92DF92EF92FF920F931F9340
:1006F000CF93DF93CDB7DEB76C970FB6F894DEBF1C
:100700000FBECDBF9C8F8B8F5B011A011F830E83A1
:100710003701C982DC0158964D915C91599741157A
:10072000510509F0E5C018968D919C9119976817AD
:1007300079070CF0CAC11A968D919C911B972816C7
:1007400039060CF0C2C18C2C912CFB0136E0C39E03
:10075000E00DF11D1124FB87EA871E161F060CF021
:10076000B4C1C40133E0880F991F3A95E1F79D8722
:100770008C87820D931D181619060CF0A6C157968A
:100780008C91811103C0203B08F02F5FAB8DBC8D95
:10079000ED91FC9111970284F385E02DCD012A8F14
:1007A00009952A8DB5E02B9F90011124F50135960E
:1007B000FF87EE87BB82AA822501A9014A195B093E
:1007C000598B488BC10108969B8B8A8BE889F989E4
:1007D000E40DF51DE258FF4F9491988761013D8229
:1007E0002C82A885A0FF13C0AB8DBC8DED91FC9130
:1007F000B981B13031F40484F585E02D2E813F813B
:1008000016C00684F785E02DEE80FF801AC0EE81C9
:10081000FF816E167F06F1F0AB8DBC8DED91FC91E2
:10082000B981B13051F40484F585E02D9301A6011E
:10083000B2018B8D9C8D09950DC00684F785E02D46
:100840007301840194014C815D816A817B818B8D70
:100850009C8D0995E885E695E887FFEFCF1ADF0ABA
:100860002C813D81280D391D3D832C834A895B896C
:10087000C416D50609F0B5CF5FEF451A550A8A812F
:100880009B81880D991D9B838A83AE85BF854A16FF
:100890005B0609F09BCFEE81FF816E167F0609F49F
:1008A000F2C0EB8DFC8DA081B181F981F13079F43A
:1008B000B5016B5F7F4F5096ED91FC91519783018D
:1008C00028E030E0A1018B8D9C8D0995DCC06A8504
:1008D0007B85681979091E96ED91FC911F9773012C
:1008E0000C851D859401A1018B8D9C8D0995CBC034
:1008F000FA0134969491329765917491291BCB013A
:10090000B7E02B9F800D911D1124FA0125913491A0
:100910003B8B2A8BFC01459154915B834A83FC01FC
:100920003296C490319654915E87329614913196E6
:10093000D4908981823058F0612E012E000C770806
:10094000AD2D0D2C000CBB0BB987A88704C01986F0
:100950001886612C712CAB8DBC8DED91FC9111979B
:100960000284F385E02DCD010995B9818B2E912C60
:10097000689CC001699C900D789C900D1124FC012D
:10098000EA0DFB1DFD87EC871C82712C612CE12F89
:10099000110FFF0B95012E0F3F1F3B872A87AC0CD1
:1009A000B11CA5014E0F5F1F5F8B4E8BC1018D0DDA
:1009B000911DD7FC9A95998F888F4E85641608F003
:1009C00062C0862D90E048855985480F591F489D83
:1009D0009001499D300D589D300D1124D901A20D73
:1009E000B31DB98BA88BAA84BB844C845D84DC8046
:1009F000BA85DB1AE88DF98DE80FF91FFD8BEC8BBA
:100A00008D2D8A0D2E893F89A216B306B9F1877004
:100A100061F48A819B810196EA89FB89AA81BB8165
:100A2000EA0FFB1F74909B838A8377FE20C0AB8DF7
:100A3000BC8DED91FC91B981B13061F40484F585F0
:100A4000E02D2E813F814C895D89B5018B8D9C8D78
:100A500009950DC00684F785E02DEE80FF808401A6
:100A6000940148895989B2018B8D9C8D0995770C29
:100A7000EFEFAE1ABE0A480C591CC2CF3C813C0DA8
:100A80003C8363949ACFAB8DBC8DED91FC91119713
:100A90000688F789E02DCD016C960FB6F894DEBF7D
:100AA0000FBECDBFDF91CF911F910F91FF90EF90BF
:100AB000DF90CF90BF90AF909F908F907F906F907E
:100AC0005F904F903F902F9009946C960FB6F894DA
:100AD000DEBF0FBECDBFDF91CF911F910F91FF9071
:100AE000EF90DF90CF90BF90AF909F908F907F90CE
:100AF0006F905F904F903F902F900895AF92BF926C
:100B0000CF92EF92FF920F931F93CF93DF93EC015D
:100B1000262F888D998D009709F040C06A3059F4CE
:100B20001D861C862C898E859F8538E0239F800D2D
:100B3000911D112441C06D3009F4AAC08E8988230B
:100B4000C1F03C898C859D8546E0349F800D911DC8
:100B5000112448855985481759075CF41D861C8661
:100B60008E859F8548E0349F800D911D11249F87BD
:100B70008E87EA88FB88088919894E855F856C8590
:100B80007D85CC88CE010E9468032C898C859D854B
:100B900036E0239F800D911D112442C06A3079F404
:100BA0001D861C862C89FC013696E4918E859F85D6
:100BB0002E9F800D911D11249F878E8769C06D30F7
:100BC00009F466C0FC0134963491631708F460C0E0
:100BD0003196E491E61708F45BC0FC013296A590CB
:100BE000B490462F50E0431B510937E0349FB001C9
:100BF000359F700D1124A60EB71EF5013296349163
:100C00003196E491332311F0E1110DC0F5013496D2
:100C1000E4912C898C859D85E29F800D911D112486
:100C20009D878C8735C0F501359644915E895523A3
:100C300011F16C89E32FF0E0E40FF11D47FDFA9507
:100C40006E9FD0016F9FB00D11244C855D854A0FBA
:100C50005B1FE885F985E417F5076CF41D861C8693
:100C6000FC013696E4918E859F856E9F800D911DC7
:100C700011249F878E87EA88FB88088919894E8509
:100C80005F856C857D85CC88CE010E946803BECFD0
:100C900081E090E0DF91CF911F910F91FF90EF9055
:100CA000CF90BF90AF9008956F927F928F929F9256
:100CB000AF92BF92CF92DF92EF92FF920F931F936A
:100CC000CF93DF93EC014B015A0169013801E881B0
:100CD000F9810284F385E02D0995E881F981028884
:100CE000F389E02D87019601A501B401CE01099594
:100CF000E881F981A501460D571D4150510902882F
:100D0000F389E02D9601B401CE010995E881F981BE
:100D10000088F189E02D9301A501B401CE01099568
:100D2000E881F981C80CD91CB601615071090088AD
:100D3000F189E02D9301A501CE010995E881F981A2
:100D40000688F789E02DCE01DF91CF911F910F9199
:100D5000FF90EF90DF90CF90BF90AF909F908F90DB
:100D60007F906F900994CF92DF92EF92FF920F9352
:100D70001F93CF93DF9300D000D000D0CDB7DEB764
:100D80006C01DC01ED91FC916217730789F4041783
:100D900015072CF4942F852FA801092F182F041B59
:100DA000150B98012F5F3F4F048CF58DE02D12C07D
:100DB0004017510709F5261737072CF4962F872F70
:100DC000B901292F382F261B370B2F5F3F4F068C79
:100DD000F78DE02D8701C601099526960FB6F89488
:100DE000DEBF0FBECDBFDF91CF911F910F91FF905E
:100DF000EF90DF90CF9008950284F385E02D2D834E
:100E00003E834B835C8369837A830995D601ED9198
:100E1000FC910488F589E02D2D813E814B815C8118
:100E200069817A81C6010995D601ED91FC91068808
:100E3000F789E02DC60126960FB6F894DEBF0FBEE7
:100E4000CDBFDF91CF911F910F91FF90EF90DF9079
:100E5000CF900994EF92FF920F931F93DC01ED91D5
:100E6000FC9111971A960D911C911B9718962D9134
:100E70003C91199700A0F1A1E02D7B0140E050E0EA
:100E800060E070E009951F910F91FF90EF90089539
:100E90004F925F926F927F928F929F92AF92BF928A
:100EA000CF92DF92EF92FF920F931F93CF93DF9336
:100EB00000D0CDB7DEB76C015A0139014801DC0121
:100EC000ED91FC910284F385E02D69837A83099585
:100ED0006981462E7A81572E640C751CD601ED91DE
:100EE000FC91461457046CF40088F189E02D8701C9
:100EF0009401A501B201C6010995BFEF4B1A5B0A27
:100F0000EDCF0688F789E02DC6010F900F90DF9195
:100F1000CF911F910F91FF90EF90DF90CF90BF90F6
:100F2000AF909F908F907F906F905F904F900994BB
:100F3000AF92BF92CF92DF92EF92FF920F931F93E7
:100F4000CF93DF9300D000D0CDB7DEB75C0169014D
:100F5000DC01ED91FC910284F385E02D4B835C83F1
:100F600069837A830995D501ED91FC9169817A8134
:100F70009B012C0D3D1D215031090488F589E02D80
:100F800078014B815C818A01C5010995D501ED91FC
:100F9000FC910688F789E02DC5010F900F900F9006
:100FA0000F90DF91CF911F910F91FF90EF90DF9005
:100FB000CF90BF90AF900994AF92BF92CF92DF9243
:100FC000EF92FF920F931F93CF93DF9300D000D047
:100FD000CDB7DEB75C016901DC01ED91FC910284C3
:100FE000F385E02D4B835C8369837A830995D50172
:100FF000ED91FC914B815C81C40ED51EB1E0CB1A02
:10100000D1080488F589E02D7801860169817A810B
:101010009B01C5010995D501ED91FC910688F789E1
:10102000E02DC5010F900F900F900F90DF91CF91A1
:101030001F910F91FF90EF90DF90CF90BF90AF90F6
:1010400009940895EF92FF920F931F93DC01ED91A5
:10105000FC9100A0F1A1E02D09951F910F91FF9047
:10106000EF9008950F931F93DC01ED91FC91068C96
:10107000F78DE02D09951F910F9108950F931F9300
:10108000DC01ED91FC91048CF58DE02D09951F910B
:101090000F910895DC01ED91FC910084F185E02D24
:1010A000099408952F923F924F925F926F927F9290
:1010B0008F929F92AF92BF92CF92DF92EF92FF9268
:1010C0000F931F93CF93DF9300D01F92CDB7DEB75E
:1010D0004C017B836A836A01590117019801241B23
:1010E000350B37FF03C0319521953109C5014A8180
:1010F0005B81841B950B97FF03C0919581959109A6
:1011000051E059838217930714F019820BC09A2D6E
:101110008B2D5801092F182F9A818B81DB82CA826F
:10112000C92ED82E8A819B81A816B9065CF49C2D05
:101130008D2D6801092F182F9A818B81BB82AA827D
:10114000A92EB82E2501AA81BB814A1A5B0A380153
:101150006C187D0877FE03C0719461947108720168
:1011600057FE03C0BFEFEB1AFB0AF594E794C016D5
:10117000D1061CF00FEF1FEF1FC001E010E01CC0F4
:10118000D401ED91FC91B9810484F585E02D9101A4
:10119000BB23C1F04A815B81B601C4010995E61801
:1011A000F708F7FE04C0C00ED11EE40CF51CEA815E
:1011B000FB813196FB83EA834A815B81A416B506E5
:1011C000FCF604C0A6016A817B81E7CF0F900F90E7
:1011D0000F90DF91CF911F910F91FF90EF90DF90D3
:1011E000CF90BF90AF909F908F907F906F905F90C7
:1011F0004F903F902F900895089580E090E00895DB
:101200001F93CF93DF93182FC8E0D0E0612F617058
:1012100086E00E949C0E61E088E00E949C0E60E0E7
:1012200088E00E949C0E1695219781F7DF91CF915F
:101230001F910895FC01838D882339F06EBD000055
:101240000DB407FEFDCF8EB5089528E030E090E89C
:10125000A5A1B6A185A5492F462319F04C91842B51
:1012600003C04C91809584238C93A7A1B0A54C9189
:1012700086A5842B8C93A7A1B0A54C9186A58095BB
:1012800084238C9396952150310911F70895089580
:101290008CBD9DBD08951F920F920FB60F92112421
:1012A0002F933F934F935F936F937F938F939F936E
:1012B000AF93BF93EF93FF9388E192E00E948C0F6E
:1012C000282F882309F460C040910602509107023C
:1012D00060910802709109028091000190910101D2
:1012E000A0910201B0910301203161F4840F951F98
:1012F000A61FB71F813826E9920728E9A207B10582
:1013000090F409C0841B950BA60BB70B8A3091058E
:10131000A105B10540F08093000190930101A093D5
:101320000201B09303018091000190910101A0910D
:101330000201B09103010B97A105B10560F48AE0A9
:1013400090E0A0E0B0E08093000190930101A093B1
:101350000201B09303018091000190910101A091DD
:101360000201B091030180389649A849B10560F0A7
:1013700080E896E9A8E9B0E080930001909301012C
:10138000A0930201B0930301FF91EF91BF91AF9140
:101390009F918F917F916F915F914F913F912F918D
:1013A0000F900FBE0F901F9018954F925F926F9203
:1013B0007F928F929F92AF92BF92CF92DF92EF92E5
:1013C000FF920F931F93CF9380911202909113027B
:1013D0008B30910508F043C0FC01EC5CFF4F0C948E
:1013E000521841E050E060E070E031C04AE050E067
:1013F00060E070E02CC042E350E060E070E027C0A5
:1014000044E650E060E070E022C044EF51E060E06C
:1014100070E01DC048EE53E060E070E018C044EC9E
:1014200059E060E070E013C048E853E160E070E02C
:101430000EC040E157E260E070E009C040EA56E8C3
:1014400061E070E004C040E251EA67E070E0409380
:101450000602509307026093080270930902880FF6
:10146000991FFC01EA5CFE4F608171816115710575
:1014700069F0FB0101900020E9F73197AF01461BAD
:10148000570B8CE092E00E94B10D14C080910C02C9
:1014900090910D02009711F00E94ED1810920D022C
:1014A00010920C02109211021092100210920F0270
:1014B00010920E02E12CF12C04E110E020EA30E061
:1014C0004FE050E060E070E08EE192E00E940B118E
:1014D00080EE9FEF909331028093300290932F0221
:1014E00080932E028AE090E090932B0280932A0250
:1014F00084E190E090932D0280932C0281E0809310
:10150000320288E691E00E94AF0DC2E0C093320241
:101510008CE390E090932B0280932A028FE090E07E
:1015200090932D0280932C02409110025091110251
:1015300060910C0270910D028EE192E00E94A70C66
:101540000CE310E020EA30E048E250E060E070E0B8
:101550008EE192E00E940B1180EE97E090933102B1
:101560008093300290932F0280932E02C093320218
:10157000C0900001D0900101E0900201F0900301C1
:1015800088EEC81683E0D806E104F104D8F58EE4AD
:1015900090E090932B0280932A0282E390E0909354
:1015A0002D0280932C028DE691E00E94AF0D809178
:1015B000000190910101A0910201B09103018436D4
:1015C0009105A105B10520F48DE691E00E94AF0DD3
:1015D00060910001709101018091020190910301DD
:1015E0004AE00E94350D8AE390E090932B028093AD
:1015F0002A028BE490E090932D0280932C028BECD6
:1016000091E060C180E4C81682E4D8068FE0E80665
:10161000F10408F0CDC088E290E090932B02809313
:101620002A0282E390E090932D0280932C0280E1C5
:10163000C81687E2D806E104F10420F48DE691E0B3
:101640000E94AF0D60910001709101018091020133
:10165000909103010E949C1520E030E04AE754E499
:101660000E945F176B017C014B015C019B01AC0187
:101670000E940C18882319F08FE691E01AC0260109
:101680003701E89477F82FEF3FEF4FE75FE7C301AB
:10169000B2010E940C1881110FC02FEF3FEF4FE7EE
:1016A0005FE7C301B2010E94971518162CF483E777
:1016B00091E00E94230D6DC02FEF3FEF4FE75FE4F5
:1016C000C701B6010E94071818161CF487E791E0BD
:1016D000F0CF2FEF3FEF4FE75FECC701B6010E945D
:1016E000971587FDF3CF20E030E0A901C701B601CF
:1016F0000E94971587FF09C08DE20E94760D460172
:101700005701B7FAB094B7F8B0942EE632E143E04F
:101710005AE3C501B4010E94F3166B017C010E94DB
:10172000D8174B015C010E949C159B01AC01C701BD
:10173000B6010E94F2166B017C014AE0C501B401BA
:101740000E94350D8EE20E94760DC4E0C15009F171
:1017500020E030E040E251E4C701B6010E94FD15EF
:101760004B015C010E94D8176B01E12CF12C4AE07F
:10177000C701B6010E94350DC701B6010E949C1534
:101780009B01AC01C501B4010E94F2166B017C0102
:10179000DDCF8AE390E090932B0280932A028BE4C2
:1017A00090E090932D0280932C0289EF91E08AC003
:1017B00089E190E090932B0280932A0282E390E0EB
:1017C00090932D0280932C02C701B60120E432E4ED
:1017D0004FE050E00E943318C9010E94810D8BE751
:1017E00091E00E94AF0DC701B60120EA36E841E062
:1017F00050E00E9433188AE0882E912CA12CB12C45
:10180000CA01B901A50194010E943318CB010E94BD
:10181000810DC701B60120E137E240E050E00E94AF
:101820003318CA01B901A50194010E943318CB01F4
:101830000E94810DC701B60128EE33E040E050E080
:101840000E943318CA01B901A50194010E943318FE
:10185000CB010E94810D8DE791E00E94AF0DC70181
:10186000B60124E630E040E050E00E943318CA019F
:10187000B901A50194010E943318CB010E94810D8A
:10188000C701B601A50194010E9433186B017C01C8
:10189000CA01B901A50194010E943318CB010E942D
:1018A000810DC6010E94810D8AE390E090932B0286
:1018B00080932A028BE490E090932D0280932C0277
:1018C0008FE791E0CF911F910F91FF90EF90DF9004
:1018D000CF90BF90AF909F908F907F906F905F90D0
:1018E0004F900C94AF0DCF92DF92EF92FF92CF9377
:1018F000DF9320E030E040E85FE40E94FD1528E23D
:101900003BE64EEE5CE40E945F170E94D1176B012C
:101910007C01C4E0D0E08C2D0E940009CD2CDE2C8F
:10192000EF2CFF24E7FCFA942197A9F780E00E94AE
:10193000000961E087E00E949C0E60E087E0DF9193
:10194000CF91FF90EF90DF90CF900C949C0ECF92B0
:10195000DF92EF92FF920F931F93CF93DF936C016F
:101960007A018B01C0E0D0E0CE15DF0589F0D80107
:101970006D918D01D601ED91FC910190F081E02DEA
:10198000C6010995892B11F47E0102C02196ECCF86
:10199000C701DF91CF911F910F91FF90EF90DF90E2
:1019A000CF900895CF92DF92EF92FF920F931F9303
:1019B000CF93DF93EC012196FC011491112309F4DC
:1019C00037C0FE0164918EE192E00E9405106E0125
:1019D000F2E0CF0ED11CFE013196C4910C2F00789D
:1019E000CF777601DC2FD15050F0F70164918EE172
:1019F00092E00E94D20FFFEFEF1AFF0AF4CFC60168
:101A00008C0F911DEC01002389F07C019FEFE91AF6
:101A1000F90AFE01649170E06F3F710511F464EF03
:101A200071E080E090E00E94080FE7011150C6CFFE
:101A3000DF91CF911F910F91FF90EF90DF90CF90AA
:101A400008950E944F1A009769F0FC010190002050
:101A5000E9F73197AF01481B590BBC018EE192E0C9
:101A60000C94A70C80E090E008958F929F92AF9223
:101A7000BF920F931F93CF93DF93CDB7DEB7A1979C
:101A80000FB6F894DEBF0FBECDBF19A2423008F4E6
:101A90004AE08E010F5D1F4F842E912CA12CB12C9A
:101AA000A50194010E941118E62FB901CA01015045
:101AB0001109EA3014F4E05D01C0E95CD801EC934F
:101AC000232B242B252B61F7C8010E94230DA196FF
:101AD0000FB6F894DEBF0FBECDBFDF91CF911F913F
:101AE0000F91BF90AF909F908F900895E0911E024C
:101AF000F0911F020190F081E02D682F8EE192E0BD
:101B00000994CF92DF92EF92FF92CF93DF936C0113
:101B1000990FEE08FF08F7FE17C08DE20E94760DC0
:101B2000EC0166277727CB016C197D098E099F0987
:101B30004AE00E94350D8C0F9D1FDF91CF91FF90E1
:101B4000EF90DF90CF9008954AE0C701B601DF9192
:101B5000CF91FF90EF90DF90CF900C94350D0C94C7
:101B6000230DEF92FF920F931F93CF93DF93EC011E
:101B70007B018A0188819981009729F02A813B8124
:101B800024173507F8F4B8016F5F7F4F0E9485195D
:101B9000009759F0998388831B830A832C813D81A8
:101BA000232B81F4FC0110820DC08881998100975C
:101BB00011F00E94ED18198218821D821C821B826E
:101BC0001A8207C01D830C83B701888199810E9406
:101BD0005D1ACE01DF91CF911F910F91FF90EF9091
:101BE0000895833081F028F4813099F08230A1F09B
:101BF00008958730A9F08830B9F08430D1F480910D
:101C000080008F7D03C0809180008F77809380005B
:101C1000089584B58F7702C084B58F7D84BD089503
:101C20008091B0008F7703C08091B0008F7D80934A
:101C3000B00008953FB7F8948091550290915602F4
:101C4000A0915702B091580226B5A89B05C02F3F1E
:101C500019F00196A11DB11D3FBFBA2FA92F982FD2
:101C60008827820F911DA11DB11DBC01CD0142E04D
:101C7000660F771F881F991F4A95D1F70895DC01D9
:101C80009B96ED91FC919C979081D0968C91892B9D
:101C900080830895DC019996ED91FC919A9790814B
:101CA0009F968C91892B80830895EF92FF920F93DA
:101CB0001F93DC01ED91FC9111971A960D911C91E7
:101CC0001B9718962D913C91199700A0F1A1E02D3A
:101CD0007B0140E050E060E070E009951F910F91BA
:101CE000FF90EF900895CF93DF93282F30E0F90114
:101CF000E258FA4F8491F901E456FA4FD491F90170
:101D0000E654FA4FC491CC2391F081110E94F10D59
:101D1000EC2FF0E0EE0FFF1FEF5BF94FA591B491B0
:101D2000EC91ED2381E090E021F480E002C080E0BE
:101D300090E0DF91CF9108951F93CF93DF93282FE9
:101D400030E0F901E258FA4F8491F901E456FA4F74
:101D5000D491F901E654FA4FC491CC23C9F0162F5F
:101D600081110E94F10DEC2FF0E0EE0FFF1FE05506
:101D7000FA4FA591B4918FB7F894111105C09C91B9
:101D8000ED2FE095E92302C0EC91ED2BEC938FBF92
:101D9000DF91CF911F910895CF93DF9390E0FC01E5
:101DA000E456FA4F2491FC01E654FA4F84918823BB
:101DB00061F190E0880F991FFC01EE56FA4FC59132
:101DC000D491FC01E055FA4FA591B491611109C07D
:101DD0009FB7F8948881209582238883EC912E23E5
:101DE0000BC0623061F49FB7F8943881822F8095E0
:101DF00083238883EC912E2B2C939FBF06C08FB733
:101E0000F894E8812E2B28838FBFDF91CF9108951E
:101E10008F929F92AF92BF92CF92DF92EF92FF92FA
:101E20006B017C010E941A0E4B015C01C114D104AC
:101E3000E104F104F1F00E941A0EDC01CB018819D3
:101E40009909AA09BB09883E9340A105B10570F321
:101E500021E0C21AD108E108F10888EE880E83E07B
:101E6000981EA11CB11CC114D104E104F10419F79E
:101E7000DDCFFF90EF90DF90CF90BF90AF909F901D
:101E80008F9008951F920F920FB60F9211242F93E7
:101E90003F938F939F93AF93BF9380915102909103
:101EA0005202A0915302B09154023091500223E0AB
:101EB000230F2D3720F40196A11DB11D05C026E882
:101EC000230F0296A11DB11D209350028093510251
:101ED00090935202A0935302B09354028091550202
:101EE00090915602A0915702B09158020196A11DFF
:101EF000B11D8093550290935602A0935702B09360
:101F00005802BF91AF919F918F913F912F910F9068
:101F10000FBE0F901F9018950F931F93CF93DF93D1
:101F2000EC018A810E94730E8C0189810E94730EDC
:101F3000000F111F802BE881EF7094E0E99FF00102
:101F40001124E80FF11DE45BFE4F808188838073CC
:101F5000DF91CF911F910F910895CF93DF93EC0103
:101F6000862F69834A8360E00E94CC0E60E08A81FC
:101F70000E94CC0E61E089810E949C0E61E08A8102
:101F80000E949C0E1882DF91CF910895DC019996F2
:101F9000ED91FC919A9790819F968C9180958923E1
:101FA000808308950F931F93CF93DF931F92CDB734
:101FB000DEB78C01FC01838D882341F080910A02F9
:101FC00090910B0269830E9448096981C801698365
:101FD0000E943F0EC8010E94C60F6981C8010E947D
:101FE0001A09C8010E944A0EF801838D882339F02E
:101FF0000F90DF91CF911F910F910C9447090F9093
:10200000DF91CF911F910F9108950F931F93CF935D
:10201000DF931F92CDB7DEB78C01DC015B968C910C
:10202000882341F080910A0290910B0269830E94FB
:1020300048096981D8019B96ED91FC919C9790810C
:10204000D0968C91809589238083C80169830E94F2
:10205000C60F6981C8010E941A09C8010E944A0E70
:10206000F801838D882339F00F90DF91CF911F9174
:102070000F910C9447090F90DF91CF911F910F9111
:102080000895611102C060E201C061E20C94051084
:102090001F93CF93DF93EC01162F66E30E94051088
:1020A000612F63706D8B8A8D6230A1F06330D1F146
:1020B000613041F0823011F0843011F460EC11C0D5
:1020C00068EC0FC0823011F0843011F460EA31C046
:1020D00068EA2FC0823011F0843011F460E001C052
:1020E00068E0CE010E94D20F8A8D813029F480E809
:1020F00090E09B878A870FC0843039F480EA90E0B3
:102100009B878A8780E590E006C080EA90E09B8705
:102110008A8780E890E09987888789A18BA38AA124
:102120008CA327C0823011F0843011F460E601C026
:1021300068E6CE010E94D20F8A8D813029F480E8B2
:1021400090E0998788870FC0843039F480EA90E066
:102150009987888780E590E006C080EA90E09987BB
:10216000888780E890E09B878A8789A18CA38AA1D1
:102170008BA3DF91CF911F910895EF92FF920F9360
:102180001F93CF93DF9300D0CDB7DEB77C01162F1E
:102190006AE229834A830E94051060E0C7010E9419
:1021A000D20FF70183A1612F680FC7010E94D20FE0
:1021B00060E0C7010E94D20FF70183A12981622F3D
:1021C000680FC7010E94D20F6BE2C7010E94051081
:1021D00060E0C7010E94D20FF70184A14A81642FF9
:1021E000680FC7010E94D20F60E0C7010E94D20FA2
:1021F000F70184A1602F680FC7010E94D20F6CE223
:10220000C7010F900F90DF91CF911F910F91FF9019
:10221000EF900C940510AF92BF92CF92DF92EF92A5
:10222000FF920F931F93CF93DF93EC015901680145
:1022300028853985621773070CF058C08A859B85FD
:10224000481759070CF052C0FB01EA0DFB1D2E1771
:102250003F071CF45901A61AB70A9A012C0D3D1D1F
:10226000821793071CF46C01C41AD50A0FEF040FF0
:102270000C0D2FEF260F2A0DCE010E94BD108B8D65
:10228000882331F080910A0290910B020E94480944
:10229000CE010E943F0ECE010E94C60F1C141D04E9
:1022A0009CF48501101611065CF46F2DCE010E947E
:1022B0001A096E2DCE010E941A0901501109F2CFA0
:1022C00081E0C81AD108EACFCE010E944A0E8B8D58
:1022D000882361F0DF91CF911F910F91FF90EF90D4
:1022E000DF90CF90BF90AF900C944709DF91CF91D2
:1022F0001F910F91FF90EF90DF90CF90BF90AF9024
:102300000895DF92EF92FF920F931F93CF93DF9385
:10231000EC017901D02E88859985681779070CF032
:1023200042C02A853B8542175307ECF59B012E0DD1
:102330003F1D821793071CF47C01E61AF70A2FEF62
:10234000260F2E0D042FCE010E94BD108B8D8823E9
:1023500031F080910A0290910B020E944809CE014F
:102360000E943F0ECE010E94C60FE114F10461F0FD
:10237000612FCE010E941A096D2DCE010E941A090B
:1023800081E0E81AF108F1CFCE010E944A0E8B8D50
:10239000882349F0DF91CF911F910F91FF90EF902B
:1023A000DF900C944709DF91CF911F910F91FF901F
:1023B000EF90DF900895DF92EF92FF920F931F93BB
:1023C000CF93DF93EC017901D02E8885998568172A
:1023D00079070CF043C08A859B8548175907F4F5A7
:1023E0009A012E0D3F1D821793071CF47C01E41AFD
:1023F000F50A8FEF840F082F0E0D262FCE010E94B5
:10240000BD108B8D882331F080910A0290910B02D0
:102410000E944809CE010E943F0ECE010E94C60FC5
:10242000E114F10461F0612FCE010E941A096D2DB3
:10243000CE010E941A0981E0E81AF108F1CFCE011D
:102440000E944A0E8B8D882349F0DF91CF911F9116
:102450000F91FF90EF90DF900C944709DF91CF919F
:102460001F910F91FF90EF90DF900895FF920F93CF
:102470001F93CF93DF93EC01122FF32E77FD36C01D
:1024800028853985621773078CF557FD2FC02A857B
:102490003B854217530754F501E0040F21E0260F56
:1024A0000E94BD108B8D882331F080910A0290919B
:1024B0000B020E944809CE010E943F0ECE010E94ED
:1024C000C60F6F2DCE010E941A09612FCE010E9406
:1024D0001A09CE010E944A0E8B8D882339F0DF91B4
:1024E000CF911F910F91FF900C944709DF91CF91ED
:1024F0001F910F91FF90089580910C0290910D0211
:102500000C94ED1880E580930A0210920B02109251
:1025100021021092200220E830E030932302209321
:10252000220280EA90E09093250280932402309367
:10253000270220932602909329028093280210926A
:10254000330210922B0210922A0210922D02109246
:102550002C0281E0809332022FEF3FEF3093310263
:102560002093300230932F0220932E028093340266
:102570001092350210923702109236022EE031E0AE
:1025800030931F0220931E029AE090933A029EE03D
:1025900090933B029FE090933C02809339028FEF2F
:1025A00080933E0280933D0240E161E18BE192E045
:1025B0000E94AD0F43E062E088E192E00E94AD0F1F
:1025C0008091000190910101A0910201B09103015D
:1025D0008093140290931502A0931602B0931702F1
:1025E000E0911202F0911302EE0FFF1FEA5CFE4F22
:1025F0006081718110920D0210920C0210920F02F4
:1026000010920E02109211021092100261157105C3
:1026100061F0FB0101900020E9F73197AF01461B03
:10262000570B8CE092E00C94B10D0895789484B52A
:10263000826084BD84B5816084BD85B5826085BDBE
:1026400085B5816085BD80916E00816080936E004C
:10265000109281008091810082608093810080913E
:1026600081008160809381008091800081608093EF
:1026700080008091B10084608093B1008091B000AF
:1026800081608093B00080917A00846080937A00AA
:1026900080917A00826080937A0080917A008160D4
:1026A00080937A0080917A00806880937A001092FB
:1026B000C10062E082E00E94CC0E62E083E00E94F2
:1026C000CC0E62E082E10E94CC0E62E084E00E94C7
:1026D000CC0E61E087E00E94CC0E61E088E00E94B1
:1026E000CC0E61E086E00E94CC0E61E085E00E94A5
:1026F000CC0E61E08FE00E94CC0E61E08EE00E9483
:10270000CC0E61E089E00E94CC0E61E089E00E947D
:10271000CC0E61E089E00E949C0E8091680084608C
:102720008093680080916D008C6080936D00789438
:102730001092400210923F02109241021092420207
:1027400061E080913B020E94CC0E61E080913A02F0
:102750000E94CC0E20913A02022E000C330BF9019C
:10276000E654FA4FE491F0E0EE0FFF1FE055FA4F08
:1027700085919491909348028093470240913B0247
:10278000042E000C550BFA01E654FA4F8491E82F01
:10279000F0E0EE0FFF1FE055FA4F85919491909372
:1027A0004A0280934902F901E456FA4FE491E0931A
:1027B0004D02FA01E456FA4FE491E0934E02809103
:1027C0003902882309F43AC0CFB7F89480914F02B8
:1027D000811127C0E4ECF5E08491E6EAF5E09491FC
:1027E000E82FF0E0EE0FFF1FEE56FA4FA591B491DF
:1027F000EC91E92321F461E08AE00E949C0E61E003
:102800008AE00E94CC0E8CB580618CBD8CB5806452
:102810008CBD61E08DE00E94CC0E61E08BE00E94F7
:10282000CC0E80914F028F5F80934F02CFBF80E527
:1028300080930A0281E080930B0249C061E080919D
:102840003E020E94CC0E61E080913D020E94CC0EBF
:1028500060E080913E020E949C0E60E080913D020B
:102860000E949C0E20913E02022E000C330BF901B7
:10287000E654FA4FE491F0E0EE0FFF1FE055FA4FF7
:1028800085919491909346028093450240913D0238
:10289000042E000C550BFA01E654FA4F8491E82FF0
:1028A000F0E0EE0FFF1FE055FA4F85919491909361
:1028B000440280934302F901E456FA4FE491E09315
:1028C0004C02FA01E456FA4FE491E0934B028EE198
:1028D00092E00E94C60F80913C028F3F21F161E09F
:1028E0000E94CC0E61E080913C020E949C0E64EF3D
:1028F00071E080E090E00E94080F60E080913C026F
:102900000E949C0E64EF71E080E090E00E94080F4E
:1029100061E080913C020E949C0E64EF71E080E0D7
:1029200090E00E94080F86E096E00E94D20C89EFAA
:1029300095E00E94D20C8EEC95E00E94D20C66E3EA
:102940008EE192E00E94051060EC8EE192E00E9420
:10295000D20F82E08093380260E08EE192E00E9424
:10296000481063E08EE192E00E9448101092340219
:1029700060E070E08EE192E00E94550E40912802E6
:10298000509129028FE090E090932B0280932A02CD
:10299000CA01449790932D0280932C0281E080938A
:1029A000320220912602309127022A5031094751E4
:1029B00051090FE110E060E070E08EE192E00E94CA
:1029C00081118FE190E090933102809330029093D7
:1029D0002F0280932E0284E891E00E94230D8AE961
:1029E00091E00E94230D8DE991E00E94AF0D61E01E
:1029F00085E00E949C0E60E085E00E949C0E61E0F4
:102A000088E00E949C0E60E088E00E949C0E61E0DD
:102A100087E00E949C0E60E087E00E949C0E0E946E
:102A2000D509C0E0D0E088EEC82E83E0D82EE12C96
:102A3000F12C8BE192E00E948C0F8823D9F0803139
:102A400049F480911202909113028A30910584F426
:102A500001960AC0803261F48091120290911302B3
:102A6000181619062CF40197909313028093120202
:102A70000E94D50982E10E94730E892B61F41092A5
:102A80001302109212020E94D50962E370E080E006
:102A900090E00E94080F84E00E94730E892BB1F42D
:102AA000C0920001D0920101E0920201F092030174
:102AB00060E070E08AE794E40E94730C0E94D509FC
:102AC0006EE571E080E090E00E94080F60910001E7
:102AD0007091010180910201909103010091140213
:102AE0001091150220911602309117020617170750
:102AF00028073907B1F00E949C150E94730C0E94B0
:102B0000D5098091000190910101A0910201B0913D
:102B100003018093140290931502A0931602B093C0
:102B20001702209709F485CF0E94000082CF0E94EF
:102B3000D91508F481E00895E89409C097FB3EF4A4
:102B400090958095709561957F4F8F4F9F4F9923FA
:102B5000A9F0F92F96E9BB279395F6958795779578
:102B60006795B795F111F8CFFAF4BB0F11F460FF38
:102B70001BC06F5F7F4F8F4F9F4F16C0882311F090
:102B800096E911C0772321F09EE8872F762F05C0A4
:102B9000662371F096E8862F70E060E02AF09A953F
:102BA000660F771F881FDAF7880F9695879597F934
:102BB0000895990F0008550FAA0BE0E8FEEF1616CE
:102BC0001706E807F907C0F012161306E407F50721
:102BD00098F0621B730B840B950B39F40A2661F095
:102BE000232B242B252B21F408950A2609F4A14038
:102BF000A6958FEF811D811D08950E9410160C94DB
:102C000081160E94731638F00E947A1620F09523E0
:102C100011F00C946A160C94701611240C94B516CD
:102C20000E94921670F3959FC1F3950F50E0551FC7
:102C3000629FF001729FBB27F00DB11D639FAA2711
:102C4000F00DB11DAA1F649F6627B00DA11D661F60
:102C5000829F2227B00DA11D621F739FB00DA11D81
:102C6000621F839FA00D611D221F749F3327A00D3B
:102C7000611D231F849F600D211D822F762F6A2FD7
:102C800011249F5750409AF0F1F088234AF0EE0F3C
:102C9000FF1FBB1F661F771F881F91505040A9F769
:102CA0009E3F510580F00C946A160C94B5165F3F58
:102CB000E4F3983ED4F3869577956795B795F795A5
:102CC000E7959F5FC1F7FE2B880F911D969587951D
:102CD00097F9089597F99F6780E870E060E008959C
:102CE0009FEF80EC089500240A9416161706180624
:102CF0000906089500240A94121613061406050600
:102D00000895092E0394000C11F4882352F0BB0F90
:102D100040F4BF2B11F460FF04C06F5F7F4F8F4FF3
:102D20009F4F089557FD9058440F551F59F05F3F2E
:102D300071F04795880F97FB991F61F09F3F79F0DD
:102D400087950895121613061406551FF2CF46955F
:102D5000F1DF08C0161617061806991FF1CF8695E1
:102D60007105610508940895E894BB2766277727C5
:102D7000CB0197F908952F923F924F925F926F92F5
:102D80007F928F929F92AF92BF92CF92DF92EF92FB
:102D9000FF920F931F93CF93DF93CDB7DEB7CA1B7C
:102DA000DB0B0FB6F894DEBF0FBECDBF09942A88A7
:102DB000398848885F846E847D848C849B84AA844F
:102DC000B984C884DF80EE80FD800C811B81AA81DC
:102DD000B981CE0FD11D0FB6F894DEBF0FBECDBFA7
:102DE000ED0108955058BB27AA270E940A170C949A
:102DF00081160E94731638F00E947A1620F039F47A
:102E00009F3F19F426F40C9470160EF4E095E7FB3E
:102E10000C946A16E92F0E94921658F3BA176207AB
:102E200073078407950720F079F4A6F50C94B4167F
:102E30000EF4E0950B2EBA2FA02D0B01B9019001D5
:102E40000C01CA01A0011124FF27591B99F0593F19
:102E500050F4503E68F11A16F040A22F232F342F61
:102E60004427585FF3CF469537952795A795F040AF
:102E70005395C9F77EF41F16BA0B620B730B840BC4
:102E8000BAF09150A1F0FF0FBB1F661F771F881F7C
:102E9000C2F70EC0BA0F621F731F841F48F48795D4
:102EA00077956795B795F7959E3F08F0B0CF9395C6
:102EB000880F08F09927EE0F9795879508950E943F
:102EC00073170C9481160E947A1658F00E9473169C
:102ED00040F029F45F3F29F00C946A1651110C94CC
:102EE000B5160C9470160E94921668F39923B1F3EC
:102EF000552391F3951B550BBB27AA276217730720
:102F0000840738F09F5F5F4F220F331F441FAA1FB3
:102F1000A9F335D00E2E3AF0E0E832D0915050406F
:102F2000E695001CCAF72BD0FE2F29D0660F771F1D
:102F3000881FBB1F261737074807AB07B0E809F003
:102F4000BB0B802DBF01FF2793585F4F3AF09E3F88
:102F5000510578F00C946A160C94B5165F3FE4F3B3
:102F6000983ED4F3869577956795B795F7959F5FCB
:102F7000C9F7880F911D9695879597F90895E1E017
:102F8000660F771F881FBB1F621773078407BA0776
:102F900020F0621B730B840BBA0BEE1F88F7E095D1
:102FA00008950E94D8176894B1110C94B51608952D
:102FB0000E949A1688F09F5798F0B92F9927B75119
:102FC000B0F0E1F0660F771F881F991F1AF0BA95CD
:102FD000C9F714C0B13091F00E94B416B1E0089561
:102FE0000C94B416672F782F8827B85F39F0B93F53
:102FF000CCF3869577956795B395D9F73EF4909580
:103000008095709561957F4F8F4F9F4F08950E94D7
:10301000D91508F48FEF08950E94D915880B990BE4
:103020000895A1E21A2EAA1BBB1BFD010DC0AA1F09
:10303000BB1FEE1FFF1FA217B307E407F50720F021
:10304000A21BB30BE40BF50B661F771F881F991F9C
:103050001A9469F760957095809590959B01AC01E5
:10306000BD01CF010895052E97FB1EF400940E9428
:103070004A1857FD07D00E94111807FC03D04EF4E0
:103080000C944A1850954095309521953F4F4F4FDD
:103090005F4F089590958095709561957F4F8F4F04
:1030A0009F4F0895EE0FFF1F0590F491E02D0994B6
:1030B000CF93DF938230910510F482E090E0E091AD
:1030C0005B02F0915C0220E030E0C0E0D0E030979D
:1030D00011F14081518148175907C0F0481759072D
:1030E00061F482819381209719F09B838A832BC09E
:1030F00090935C0280935B0226C02115310519F084
:103100004217530718F49A01BE01DF01EF01028054
:10311000F381E02DDCCF2115310509F1281B390B96
:103120002430310590F412968D919C91139761157E
:10313000710521F0FB019383828304C090935C02AC
:1031400080935B02FD01329644C0FD01E20FF31F44
:1031500081939193225031092D933C933AC0209151
:10316000590230915A02232B41F4209106013091EB
:10317000070130935A0220935902209104013091A3
:1031800005012115310541F42DB73EB740910801E5
:1031900050910901241B350BE0915902F0915A021C
:1031A000E217F307A0F42E1B3F0B2817390778F01E
:1031B000AC014E5F5F4F2417350748F04E0F5F1F7D
:1031C00050935A02409359028193919302C0E0E0D8
:1031D000F0E0CF01DF91CF9108950F931F93CF932C
:1031E000DF93009709F48CC0FC013297138212829E
:1031F00000915B0210915C020115110581F42081A0
:103200003181820F931F2091590230915A02281761
:10321000390779F5F0935A02E093590271C0D80149
:1032200040E050E0AE17BF0750F412962D913C914C
:103230001397AD012115310509F1D901F3CF9D0196
:10324000DA013383228360817181860F971F821791
:10325000930769F4EC0128813981260F371F2E5F0F
:103260003F4F318320838A819B8193838283452BC7
:1032700029F4F0935C02E0935B0242C01396FC9346
:10328000EE931297ED01499159919E01240F351F3C
:10329000E217F30771F480819181840F951F0296E4
:1032A00011969C938E938281938113969C938E9317
:1032B0001297E0E0F0E0D80112968D919C9113975F
:1032C000009719F0F8018C01F6CF8D919C9198012F
:1032D0002E5F3F4F820F931F2091590230915A0267
:1032E0002817390769F4309729F410925C0210927C
:1032F0005B0202C01382128210935A020093590299
:10330000DF91CF911F910F910895A0E0B0E0EBE81D
:10331000F9E10C94BF16EC01009721F4CB010E9457
:103320005818B8C0FC01E60FF71F9C012250310964
:10333000E217F30708F4ACC0D9010D911C91119765
:1033400006171707B0F00530110508F49FC0C80133
:1033500004978617970708F499C002501109061BB5
:10336000170B019311936D937C93CF010E94ED187D
:103370008DC05B01A01AB10A4C01800E911EA09174
:103380005B02B0915C0240E050E0E12CF12C109720
:1033900009F44AC0A815B905D1F56D907C90119734
:1033A000630182E0C80ED11CCA14DB0480F1A301C2
:1033B0004A195B096A0182E0C80ED11C1296BC90C2
:1033C00012971396AC91B5E0CB16D10440F0B282BF
:1033D000A38351834083D9016D937C930AC00E5F10
:1033E0001F4FC301800F911FF90191838083EB2D43
:1033F000FA2FE114F10431F0D7011396FC93EE9308
:10340000129744C0F0935C02E0935B023FC08D9141
:103410009C9111974817590708F4AC017D01129649
:103420000D90BC91A02DB3CF8091590290915A027A
:1034300088159905E1F446175707C8F480910401EF
:1034400090910501009741F48DB79EB74091080116
:1034500050910901841B950BE817F907C8F4F09304
:103460005A02E0935902F901718360830FC0CB01C6
:103470000E9458187C01009759F0A801BE010E94D3
:10348000541ACE010E94ED18C70104C0CE0102C03B
:1034900080E090E0CDB7DEB7EEE00C94DB1681E083
:1034A00090E0F8940C94641AFB01DC0102C00190D6
:1034B0000D9241505040D8F70895FB01DC01019076
:1034C0000D920020E1F7089513E0C7E2D3E004C0B5
:1034D000FE010E9452182196C832D107C9F7F8940C
:0234E000FFCF1C
:1034E200E803000000005D028000000000007E058D
:1034F200A70CFD08FC08361251084A0822083E08AB
:1035020032085208210848104110DB1181110B11B9
:10351200550EB3065406B301BA01C101C801CF0169
:10352200D601DE01E601EE01F601FE010002040011
:103532000300011003020000030201000600040060
:103542000605002006050400537465703A20006EDB
:10355200616E00696E66006F7666002E002C002098
:103562004D487A00414439383530203120487A209C
:10357200746F2035204D487A20000D0A002020204B
:1035820073696E65776176652067656E65726174D1
:103592006F720020203120487A0020313020487A92
:1035A2000020353020487A0031303020487A00350A
:1035B200303020487A00202031206B487A00322EA9
:1035C20035206B487A00202035206B487A00203164
:1035D20030206B487A00313030206B487A00353029
:0635E20030206B487A0066
:107800000C94343C0C94513C0C94513C0C94513CE1
:107810000C94513C0C94513C0C94513C0C94513CB4
:107820000C94513C0C94513C0C94513C0C94513CA4
:107830000C94513C0C94513C0C94513C0C94513C94
:107840000C94513C0C94513C0C94513C0C94513C84
:107850000C94513C0C94513C0C94513C0C94513C74
:107860000C94513C0C94513C11241FBECFEFD8E036
:10787000DEBFCDBF11E0A0E0B1E0ECE9FFE702C060
:1078800005900D92A230B107D9F712E0A2E0B1E065
:1078900001C01D92AD30B107E1F70E942D3D0C945F
:1078A000CC3F0C94003C982F959595959595959582
:1078B000905D8F708A307CF0282F295A8091C0000B
:1078C00085FFFCCF9093C6008091C00085FFFCCF60
:1078D0002093C6000895282F205DF0CF982F809127
:1078E000C00085FFFCCF9093C6000895EF92FF92F1
:1078F0000F931F93EE24FF2487018091C00087FD22
:1079000017C00894E11CF11C011D111D81E4E8164B
:1079100082E4F8068FE0080780E0180770F3E09132
:107920000401F091050109958091C00087FFE9CF1E
:107930008091C6001F910F91FF90EF9008950E94D3
:10794000763C982F8091C00085FFFCCF9093C600B5
:1079500091362CF490330CF09053892F089597555D
:10796000892F08951F930E949F3C182F0E949F3CCF
:107970001295107F810F1F9108951F93182F882350
:1079800021F00E94763C1150E1F71F9108951F935A
:10799000182F0E94763C803249F0809103018F5F5E
:1079A000809303018530C1F01F9108958091C0003C
:1079B00085FFFCCF84E18093C6008091C00085FFE5
:1079C000FCCF1093C6008091C00085FFFCCF80E102
:1079D0008093C6001F910895E0910401F091050184
:1079E00009951F9108950E94763C803241F0809164
:1079F00003018F5F80930301853081F008958091AA
:107A0000C00085FFFCCF84E18093C6008091C00058
:107A100085FFFCCF80E18093C6000895E0910401CA
:107A2000F09105010995089540E951E08823A1F0FE
:107A30002D9A28EE33E0FA013197F1F721503040CA
:107A4000D1F72D9828EE33E0FA013197F1F7215064
:107A50003040D1F7815061F708953F924F925F9285
:107A60006F927F928F929F92AF92BF92CF92DF924E
:107A7000EF92FF920F931F93CF93DF93000080E16B
:107A80008093C4001092C50088E18093C10086E015
:107A90008093C2005098589A259A81E00E94143D24
:107AA00024E1F22E9EE1E92E85E9D82E0FE0C02ECA
:107AB00010E1B12EAA24A394B1E49B2EA6E58A2E50
:107AC000F2E57F2EE0E26E2E79E4572E63E5462E36
:107AD00050E5352E0E94763C8033B1F18133B9F107
:107AE000803409F46FC0813409F476C0823409F41B
:107AF00085C0853409F488C0803531F1823521F1A3
:107B0000813511F1853509F485C0863509F48DC0BC
:107B1000843609F496C0843709F403C1853709F423
:107B200072C1863709F466C0809103018F5F80932C
:107B30000301853079F6E0910401F0910501099582
:107B40000E94763C803351F60E94F33CC3CF0E94E2
:107B5000763C803249F78091C00085FFFCCFF092DF
:107B6000C6008091C00085FFFCCF9092C600809136
:107B7000C00085FFFCCF8092C6008091C00085FFC9
:107B8000FCCF7092C6008091C00085FFFCCF609250
:107B9000C6008091C00085FFFCCF5092C600809146
:107BA000C00085FFFCCF4092C6008091C00085FFD9
:107BB000FCCF3092C6008091C00085FFFCCFB09210
:107BC000C60088CF0E94763C863808F4BDCF0E945C
:107BD000763C0E94F33C7ECF0E94763C803809F4CC
:107BE0009CC0813809F40BC1823809F43CC1883942
:107BF00009F48FC080E00E94C73C6CCF84E10E94F2
:107C0000BD3C0E94F33C66CF85E00E94BD3C0E94D3
:107C1000F33C60CF0E94763C809306010E94763C44
:107C2000809307010E94F33C55CF0E94763C80333D
:107C300009F41DC183E00E94BD3C80E00E94C73C66
:107C400049CF0E94763C809309020E94763C809343
:107C5000080280910C028E7F80930C020E94763C79
:107C6000853409F415C18091080290910902892B8D
:107C700089F000E010E00E94763CF801E85FFE4FDA
:107C800080830F5F1F4F80910802909109020817AF
:107C9000190788F30E94763C803209F045CF809125
:107CA0000C0280FF01C16091060170910701660F0F
:107CB000771F7093070160930601A0910802B091AD
:107CC00009021097C9F0E8E0F1E09B01AD014E0F09
:107CD0005F1FF999FECF32BD21BD819180BDFA9A17
:107CE000F99A2F5F3F4FE417F50799F76A0F7B1F4B
:107CF00070930701609306018091C00085FFFCCF5F
:107D0000F092C6008091C00085FFFCCFB092C60003
:107D1000E1CE83E00E94C73CDDCE82E00E94C73CFA
:107D2000D9CE0E94763C809309020E94763C8093D3
:107D300008028091060190910701880F991F909386
:107D40000701809306010E94763C853409F4A6C0A1
:107D500080910C028E7F80930C020E94763C8032D0
:107D600009F0B8CE8091C00085FFFCCFF092C6002C
:107D7000609108027091090261157105B9F140E046
:107D800050E080910C02A82FA170B82FB27011C0E2
:107D9000BB2309F45CC0E0910601F0910701319624
:107DA000F0930701E09306014F5F5F4F46175707B7
:107DB000E8F4AA2369F3F999FECF209106013091E6
:107DC000070132BD21BDF89A90B58091C00085FFB2
:107DD000FCCF9093C6002F5F3F4F30930701209355
:107DE00006014F5F5F4F4617570718F38091C00099
:107DF00085FDE5CE8091C00085FFF8CFE0CE81E023
:107E00000E94C73C67CE0E94763C803209F08CCE3F
:107E10008091C00085FFFCCFF092C6008091C00029
:107E200085FFFCCFE092C6008091C00085FFFCCFAB
:107E3000D092C6008091C00085FFFCCFC092C600E2
:107E40008091C00085FFFCCFB092C60043CEE09188
:107E50000601F091070194918091C00085FFFCCF4D
:107E60009093C6009CCF80E10E94C73C33CE0E9415
:107E7000763C0E94763C182F0E94763C112309F430
:107E800083C0113009F484C08FE00E94C73C22CE29
:107E900080910C02816080930C02E5CE80910C02EF
:107EA000816080930C0259CF809107018823880F4D
:107EB000880B8A2180930B02809106019091070123
:107EC000880F991F90930701809306018091080203
:107ED00080FF09C080910802909109020196909359
:107EE000090280930802F894F999FECF1127E091D6
:107EF0000601F0910701C8E0D1E08091080290915D
:107F00000902103091F40091570001700130D9F34B
:107F100003E000935700E89500915700017001308D
:107F2000D9F301E100935700E89509901990009169
:107F3000570001700130D9F301E000935700E89534
:107F40001395103498F011270091570001700130FB
:107F5000D9F305E000935700E895009157000170B0
:107F60000130D9F301E100935700E895329602976A
:107F700009F0C7CF103011F00296E5CF112480919F
:107F8000C00085FFB9CEBCCE8EE10E94C73CA2CD19
:0C7F900085E90E94C73C9ECDF894FFCF0D
:027F9C00800063
:040000030000780081
:00000001FF
